:020000040000fa
:080000006e0404000000000082
:020000040000fa
:020000040002f8
:04afe000dfff00008f
:020000040000fa
:020000040002f8
:04afe400ffff00006b
:020000040000fa
:020000040002f8
:04afe80078ff0000ee
:020000040000fa
:020000040002f8
:04afec007dff0000e5
:020000040000fa
:020000040002f8
:04aff00078ff0000e6
:020000040000fa
:1000080000000000000000000000000000000000e8
:10001800660400000000000000000000000000006e
:10002800000000000000000000000000320800008e
:1000380000000000000000000000000000000000b8
:100048007208000000000000000000001e09000007
:100058008e090000ba09000000000000000000003e
:100068000000000000000000000000000000000088
:100078000000000000000000000000000000000078
:100088000000000000000000000000009e080000c2
:10009800de08000000000000000000000000000072
:1000a8000000000000000000000000000000000048
:1000b8000000000000000000000000000000000038
:1000c8000000000000000000000000000000000028
:1000d8000000000000000000000000000000000018
:1000e8000000000000000000000000000000000008
:1000f80000000000000000000000000000000000f8
:1001080000000000000000000000000000000000e7
:1001180000000000000000000000000000000000d7
:100128000000000056090000000000000000000068
:1001380000000000000000000000000000000000b7
:1001480000000000000000000000000000000000a7
:100158000000000000000000000000000000000097
:100168000000000000000000000000000000000087
:100178000000000000000000000000000000000077
:100188000000000000000000000000000000000067
:100198000000000000000000f8090000240a000028
:1001a800500a0000000000000000000000000000ed
:1001b8000000000000000000000000000000000037
:1001c8000000000000000000000000000000000027
:1001d8000000000000000000000000000000000017
:1001e8000000000000000000000000000000000007
:1001f80000000000000000000000000000000000f7
:1002080000000000000000000000000000000000e6
:1002180000000000000000000000000000000000d6
:1002280000000000000000000000000000000000c6
:1002380000000000000000000000000000000000b6
:1002480000000000000000000000000000000000a6
:100258000000000000000000000000000000000096
:100268000000000000000000000000000000000086
:0c0278000000000000000000000000007a
:020000040000fa
:10040000803e2000030007008100e900fcff3a0065
:1004100000000600831f7800c20320000400bc0017
:1004200066015100e0815900f23fb1000380b10044
:1004300006003500ee03090000000000423fb10055
:100440000380b100fbff3d001200b000223fb0006e
:10045000020035000280090000000000cf01780092
:1004600000000600869fbe00889fbe008a9fbe00d7
:100470008c9fbe00c10007000301330003866c009f
:100480006450e1002e0032006420e10033003200ad
:100490006150e1002f0032006120e10031003200a4
:1004a00085855500eb07b0000900200008042000f6
:1004b000050037000804440089844c000a0031001c
:1004c0000603430087834b000001530081815b00da
:1004d000f8ff33000203be000800a0000804440037
:1004e00089844c00f6ff3900c639dd0083017300b2
:1004f00001003200130020008904d1000884d300d9
:100500000998a300050032000800a7000300a0001e
:100510008904d1000884d3008b05e8008904d10048
:100520000884d3000001eb000281d200b000070074
:1005300001f0a1000cf0a70001f0a000db003700e3
:100540006420e100de0032000801be000200be00af
:10055000f7ff37006120e100d90032006000b800e9
:10056000f3ff37000000200001f82700f0ff3700fc
:10057000869fbe00889fbe008a9fbe008c9fbe00e3
:100580007e000700c000330003866c006450e10069
:10059000240032006420e100270032006150e100b5
:1005a000220032006120e100210032008b854200f0
:1005b000eb07b1000134b800003ab800080442006b
:1005c00089844a00013ab8000030b80088804000b1
:1005d00009014a0004003300000040008180480007
:1005e000020149008b05e900c909dd0083017000a3
:1005f0000100320013002000c814de004814dd00a2
:100600004709de001200b200c808de00088470004e
:100610007700070001f0a1000cf0a70001f0a00096
:10062000a20037006120e100a50032000801be00f1
:100630000200be00f7ff37006150e100fcff3a0006
:100640009f003700829fbe000001be0053000700dc
:100650000470a70003f0a10003f8a30015003a00fe
:100660006509b100110032000a0035006928e10077
:1006700003003500010028004f01be000000050006
:1006800000004000818048008502e900fcff3a003c
:1006900006003700f88f4200060035008100d100c7
:1006a0000080d3008502e800fcff3a004f01be0045
:1006b000000006008000eb004f01be0000000500b6
:1006c0000080fb008000eb00829fbe00889fbe0080
:1006d0008a9fbe00010578000100e000040035009b
:1006e00008003c000000e000200032000500370058
:1006f00060001000e080180002003b0001f02400c0
:100700001a0037000004be006011b8006b09200019
:100710000982cf00020039000882cf000441b000f6
:10072000694252000e00320008003b0082817100d5
:10073000610164008904d1000884d3008b05e800be
:100740000442e800f9ff3a000500370008044400bd
:1007500089844c008b05e9000442e900fbff3a0064
:10076000230007000af0a70001f0a0004f05be001b
:100770004f04be004f01be00000006000004be0092
:10078000060007000003be000405be000200be0014
:1007900002000700844f750000000600c70ade0053
:1007a000f107b200f50fb20008003200e1cf4200bd
:1007b000020032000170a00024000500810f7000cb
:1007c000010032000408050044000500810f70009c
:1007d00002003a00140005008502e9000000400014
:1007e00081c04800fcff3b000170a0002400050010
:1007f00081002000618055000b003d000b002000af
:1008000061fe2f000100e1001d00340082817100b3
:10081000610164008904d1000884d3000000e8006d
:10082000faff3a00710020006100640003007000cc
:10083000020060000900320061044400e0844c00c2
:100840000988a500050032008b05e8006808e10072
:1008500002003a008904d1000884d300f20f20007e
:100860000258e10005003d00c75ddd00f907b20058
:100870008980750008007800000006000bf827004a
:100880008b007800000005000200be006450e1000b
:10089000050036006420e100020036000968a3006c
:1008a00001003a000800be000160a0004f06be0033
:1008b0004f05be004f04be004f03be0000000600ff
:1008c000f0ff2f00f1ff2700f8ff37000020ef00b6
:1008d0000220ef00c088a900004006000f002100a0
:1008e000b02e210000018800000000000000eb0095
:1008f000000778000c000900002f78000007eb00cb
:100900005420ef000e2eef001e2eef000000eb0033
:10091000a1212100e51d09008018780040a7a90049
:10092000a1002000b6fe0700e0022000303a880057
:1009300044e7a90044c7a9004407a9004427a90027
:100940004447a9004467a9004487a900300020005b
:100950000600fc003174200082072000a30920005b
:10096000824878008348780080487800113a8000f7
:10097000618070000600fc002174200062042000e9
:10098000730520008248780083487800804878000a
:100990004427ef00e0022000303a880030002000b9
:1009a0000d00fc003174200082072000a309200004
:1009b0008248780083487800804878000000200052
:1009c0002174200062042000730520008248780012
:1009d000834878008048780042a7ae00feff3700c9
:1009e000813e200086fe070010c0b30086e6b700f7
:1009f00090c2b300c4e6b700100220000070880067
:100a0000007025008070880010aea90010cea900eb
:100a10004188a80041a8a90041c8a80004a1a800d5
:100a20000481a90005e1a8000068a9001061a800e0
:100a30001021a90011e1a80011a1a90010a1a8008e
:100a40001081a8000621ef000a21ef000ca1ef00a1
:100a50000ea1ef004408a8004428a9004448a900ba
:100a60000108a9002108a8001fe1a8001fa1a900f2
:100a70001ec1a9001ea1a8001e81a9001e61a90017
:100a80001e21a9004d88a8004da8a9004dc8a800a6
:100a90000368a90021e1a80021a1a90020c1a900a3
:100aa00020a1a8002081a9002021a9004e08a800ab
:100ab0004e28a9004e48a8000388a9002002a900da
:100ac0002022a9002042a90020a2a9002062a9009a
:100ad0002082a90020e2a9002102a9002122a90068
:100ae000700720004011880022a2a90022c2a9009c
:100af00022e2a90021e2a8002182a9004588a900dc
:100b000045a8a80045c8a8002168a8002828a80072
:100b100023e2a90023e2a9002342a8002362a9003e
:100b20000188a9002188a8004608a8004628a80036
:100b30004648a9002bc8a9002be8a9002c08a90049
:100b40000bc8a9000be8a9000c08a90001eca9003a
:100b500001aca900016ca900014ca800012ca9005e
:100b6000010ca90000eca900008ca90000aca900b0
:100b700000cca900000ca900002ca900004ca90081
:100b8000006ca900202cef00402cef00602cef003f
:100b90000040200020608800020ca900022ca9005f
:100ba000024ca900262cef00462cef00662cef002b
:100bb000282cef00482cef00682cef000aacef0067
:100bc00023eca80023cca90043eca80043cca90047
:100bd00063eca80063cca900dabc2a001b32240015
:100be00030002c00fa608800fb60880020618800db
:100bf000dabc2a001b32240000002800fa608800ba
:100c0000fb60880010618800dabc2a001b322400d7
:100c100030002c00fa608800fb60880020628800a9
:100c2000dabc2a001b32240000002800fa60880089
:100c3000fb60880010628800dabc2a001b322400a6
:100c400030002c00fa608800fb6088002063880078
:100c5000dabc2a001b32240000002800fa60880059
:100c6000fb6088001063880011eea90011aea90096
:100c7000116ea900a70037003f00370000202000b8
:100c80000061880000202000006288000020200011
:100c900000638800020ca900022ca800024ca800e6
:100ca00004acef0028acef0048acef0068acef00fc
:100cb000262cef00462cef00662cef000aacef006c
:100cc00023eca80023cca90043eca80043cca90046
:100cd00063eca80063cca900dabc2a001b32240014
:100ce00030002c00fa608800fb60880020618800da
:100cf000dabc2a001b32240000002800fa608800b9
:100d0000fb60880010618800dabc2a001b322400d6
:100d100030002c00fa608800fb60880020628800a8
:100d2000dabc2a001b32240000002800fa60880088
:100d3000fb60880010628800dabc2a001b322400a5
:100d400030002c00fa608800fb6088002063880077
:100d5000dabc2a001b32240000002800fa60880058
:100d6000fb6088001063880011eea90011aea90095
:100d7000116ea90067003700350037000010200011
:100d80000061880000102000006288000010200030
:100d900000638800020ca900022ca800024ca800e5
:100da0000a2cef0004acef00282cef005055250072
:100db00040628800a0aa2a0040638800dabc2a00aa
:100dc0001b32240030002c00fa608800fb60880091
:100dd00020618800dabc2a001b32240000002c00ad
:100de000fa608800fb60880010618800dabc2a0085
:100df0001b32240030002c00fa608800fb60880061
:100e000020628800dabc2a001b32240000002c007b
:100e1000fa608800fb60880010628800dabc2a0053
:100e20001b32240030002c00fa608800fb60880030
:100e300020638800dabc2a001b32240000002c004a
:100e4000fa608800fb60880010638800310037007a
:100e500030003700001020000061880000102000e2
:100e600000628800020ca900022ca800024ca80015
:100e70000a2cef0004acef00282cef000000240047
:100e800040628800dabc2a001b32240030002c00ab
:100e9000fa608800fb60880020618800dabc2a00c4
:100ea0001b32240000002c00fa608800fb608800e0
:100eb00010618800dabc2a001b32240030002c00ac
:100ec000fa608800fb60880020628800dabc2a0093
:100ed0001b32240000002c00fa608800fb608800b0
:100ee00010628800dabc2a001b32240030002c007b
:100ef000fa608800fb60880020638800dabc2a0062
:100f00001b32240000002c00fa608800fb6088007f
:100f100010638800218ca900418ca900618ca90074
:100f2000216ca900416ca900616ca900214ca900a9
:100f3000414ca900614ca90020eca80040eca8009d
:100f400060eca8003e2cef005e2cef007e2cef0042
:100f500001eca8000000eb00e19e2100ff00090069
:100f600080587800a372ef00a472ef007632ef0091
:100f70007832ef002232ef000000eb00e1ae2100fa
:100f80000801090080587800a572ef00a672ef00f2
:100f90000080eb00e19c21000f0009008018780020
:100fa0000000eb00e14c2100ff00090080187800f0
:100fb000c072ef00c172ef008d0807009d0a0700a4
:100fc000710b070080d92100d0918800f007200024
:100fd000e091880020632100f091880060052000e6
:100fe00000928800e04f2200109288007e32ef00cd
:100ff00000f023000094880080d92100209288000e
:10100000f007200030928800206321004092880081
:101010006005200050928800e04f22006092880016
:101020008232ef0000f023002094880080d9210054
:1010300070928800f00720008092880020632100d1
:101040009092880060052000a0928800e04f220066
:10105000b09288008632ef0000f0230040948800b0
:1010600032013700ff3ffc004200f8003600f80074
:101070004400f8008e1f78000e0020000d000900cb
:10108000be1f78003200f8000100fc000068a900d3
:101090000021ef0013eeaf000400370050938000f2
:1010a0001008880015eea800030037006093800048
:1010b0001008880015eea900ff3ffc003200f9007f
:1010c000ae0120000d0009004f1778004f0778008f
:1010d0004400f9003600f9004200f9000100fc006c
:1010e00000400600ff3ffc004200f8003600f80018
:1010f0004400f8008e1f78000e0020000d0009004b
:10110000be1f78003200f8000100fc000108a900b1
:10111000ff3ffc003200f900ae0120000d00090085
:101120004f1778004f0778004400f9003600f900a7
:101130004200f9000100fc0000400600ff3ffc00f7
:101140004200f8003600f8004400f8008e1f7800d6
:101150000e0020000d000900be1f78003200f800cc
:101160000100fc000368a9001421ef0013aeaf00da
:101170000400370070938000d008880015aea800e6
:101180000300370080938000d008880015aea900c6
:10119000ff3ffc003200f900ae0120000d00090005
:1011a0004f1778004f0778004400f9003600f90027
:1011b0004200f9000100fc0000400600ff3ffc0077
:1011c0004200f8003600f8004400f8008e1f780056
:1011d0000e0020000d000900be1f78003200f8004c
:1011e0000100fc000388a9001821ef00136eaf0076
:1011f0000400370090938000e0088800156ea80076
:1012000003003700a0938000e0088800156ea90055
:10121000ff3ffc003200f900ae0120000d00090084
:101220004f1778004f0778004400f9003600f900a6
:101230004200f9000100fc0000400600ff3ffc00f6
:101240004200f8003600f8004400f8008e1f7800d5
:101250000e0020000d000900be1f78003200f800cb
:101260000100fc000168a900a372ec00a3d2bf003a
:101270008080fb0030118000e29e210080707900a8
:10128000ff3ffc003200f900ae0120000d00090014
:101290004f1778004f0778004400f9003600f90036
:1012a0004200f9000100fc0000400600ff3ffc0086
:1012b0004200f8003600f8004400f8008e1f780065
:1012c0000e0020000d000900be1f78003200f8005b
:1012d0000100fc000828a9002242af00048ea800eb
:1012e0002222ae000200370014eea8002222a9003c
:1012f000ff3ffc003200f900ae0120000d000900a4
:101300004f1778004f0778004400f9003600f900c5
:101310004200f9000100fc0000400600ff3ffc0015
:101320004200f8003600f8004400f8008e1f7800f4
:101330000e0020000d000900be1f78003200f800ea
:101340000100fc000188a900ff3ffc003200f90009
:10135000ae0120000d0009004f1778004f077800fc
:101360004400f9003600f9004200f9000100fc00d9
:1013700000400600ff3ffc004200f8003600f80085
:101380004400f8008e1f78000e0020000d000900b8
:10139000be1f78003200f8000100fc0001a8a9007f
:1013a000c072ec00c0d2bf000080fb000000400013
:1013b000e14c21000218800002b07800022eaa0041
:1013c000002ea900ff3ffc003200f900ae01200012
:1013d0000d0009004f1778004f0778004400f9000e
:1013e0003600f9004200f9000100fc000040060050
:1013f000ff3ffc004200f8003600f8004400f8000f
:101400008e1f78000e0020000d000900be1f78001e
:101410003200f8000100fc000bc8a900ff3ffc00ef
:101420003200f900ae0120000d0009004f177800ce
:101430004f0778004400f9003600f9004200f90037
:101440000100fc0000400600ff3ffc004200f800e5
:101450003600f8004400f8008e1f78000e002000cf
:101460000d000900be1f78003200f8000100fc00ea
:101470000be8a900ff3ffc003200f900ae0120009c
:101480000d0009004f1778004f0778004400f9005d
:101490003600f9004200f9000100fc00004006009f
:1014a000ff3ffc004200f8003600f8004400f8005e
:1014b0008e1f78000e0020000d000900be1f78006e
:1014c0003200f8000100fc000c08a900ff3ffc00fe
:1014d0003200f900ae0120000d0009004f1778001e
:1014e0004f0778004400f9003600f9004200f90087
:1014f0000100fc0000400600a4d2bf00a352e3009c
:1015000007003200a472ec00a4d2bf000080fb00f0
:10151000e19e210060c07800a7f2b700010037000b
:10152000a7f2ef000000060000000600300880006f
:10153000b093880050088000c0938800eeff070039
:10154000d0ceb300a752b50006003900e0cfb300fb
:10155000a752b5000100390001003700a872ef0062
:1015600048033700a7f2ae0037003700a872ef003b
:10157000c0c8b300a752e30005003a00a7d2bf00dd
:10158000a8f2b700a9f2ef00aaf2ef002d00370091
:10159000c0c9b300a752e30005003a00a7d2bf00bc
:1015a000a8f2b700abf2ef00acf2ef002500370075
:1015b000c0cab300a752e30005003a00a7d2bf009b
:1015c000a8f2b700adf2ef00aef2ef001d00370059
:1015d000c0cbb300a752e30005003a00a7d2bf007a
:1015e000a8f2b700aff2ef00b0f2ef00150037003d
:1015f000c0ccb300a752e30004003a00a7d2bf005a
:10160000a8f2b700b1f2ef000e003700c0cdb30072
:10161000a752e30004003a00a7d2bf00a8f2b70027
:10162000b2f2ef0007003700c0ceb300a752e300cc
:1016300004003a00a7d2bf00a8f2b700b3f2ef004f
:10164000b4f2ef000f033700a852e20002003a00a4
:101650000c0337000b033700c0c8b300a852e300e7
:10166000be003a0000e0ef00a952e30003003a0098
:10167000a7d2bf00a9f2b700b7003700a7d2bf00ba
:10168000aaf2b700a952e20008003a00100ea90021
:10169000140ea9002612a9002412a900ceb9ef0049
:1016a000d0b9ef00b732a800aa00370010c0b300cd
:1016b000a952e30008003a00102ea900142ea90038
:1016c0002632a9002432a900d2b9ef00d4b9ef0024
:1016d000b732a8009f00370020c0b300a952e30032
:1016e00008003a00108ea900148ea9002652a90005
:1016f0002452a900d6b9ef00d8b9ef00b732a8003c
:101700009400370030c0b300a952e30008003a004b
:10171000008ea900048ea9002672a9002472a900d7
:10172000dab9ef00dcb9ef00b732a8008900370062
:1017300040c0b300a952e30003003a0010cea90054
:1017400014cea9008300370050c0b300a952e300b3
:1017500003003a0010eea90014eea9007d00370046
:10176000a9d2bf0051c1b30080cf100026003600bf
:1017700090c3b300a952e30023003e00c872ef00fb
:10178000aa52e20003003600aad2bf000080fb008c
:10179000109288004212e20013003600c8d2a8005e
:1017a0004012ec00d090880010928000d29080000f
:1017b0000200e00002003200110009000280d8009f
:1017c000e0928800e0928000b2938000c393800092
:1017d00000004100e08049000001be00f2ce880018
:1017e00003cf880006003700deb9ef00e0b9ef0054
:1017f000262cef002068a9000068a90015eea900ba
:10180000b732a80053003700a9d2bf0091c3b3007c
:1018100080cf100026003600d0c5b300a952e300e7
:1018200023003e00ca72ef00aa52e2000300360015
:10183000aad2bf000080fb00609288004c12e20038
:1018400013003600cad2a8004a12ec00d0908800db
:1018500060928000d29080000200e000020032001e
:10186000110009000280d8001093880010938000b6
:10187000b2938000c393800000004100e0804900e3
:101880000001be0012cf880023cf88000600370079
:10189000e2b9ef00e4b9ef00462cef002368a9009d
:1018a0000368a90015aea900b732a80029003700c7
:1018b000a9d2bf00d1c5b30080cf100025003600eb
:1018c000f0c7b300a952e30022003e00cc72ef0043
:1018d000aa52e20003003600aad2bf000080fb003b
:1018e000b09288005612e20013003600ccd2a80055
:1018f0005412ec00d0908800b0928000d29080000a
:101900000200e00002003200110009000280d8004d
:101910004093880040938000b2938000c39380007e
:1019200000004100e08049000001be0032cf880085
:1019300043cf880006003700e6b9ef00e8b9ef00b2
:10194000662cef002388a9000388a900156ea90062
:10195000b732a800a9f2ef004a023700c0c9b300ad
:10196000a852e3000d023a0000e0ef00ab52e300a2
:1019700003003a00a7d2bf00abf2b700060237005f
:10198000a7d2bf00acf2b700ac52e200a6003a000a
:10199000ab52e20008003a00100ea900140ea90094
:1019a0002612a9002412a900ceb9ef00d0b9ef0089
:1019b000b732a8009b00370010c0b300ab52e30061
:1019c00008003a00102ea900142ea9002632a90002
:1019d0002432a900d2b9ef00d4b9ef00b732a80081
:1019e0009000370020c0b300ab52e30008003a007b
:1019f000108ea900148ea9002652a9002452a90015
:101a0000d6b9ef00d8b9ef00b732a800850037008b
:101a100030c0b300ab52e30008003a00008ea900ca
:101a2000048ea9002672a9002472a900dab9ef0079
:101a3000dcb9ef00b732a8007a00370040c0b3002d
:101a4000ab52e30003003a0010cea90014cea90067
:101a50007400370050c0b300ab52e30003003a00fb
:101a600010eea90014eea9006e003700abd2bf0043
:101a700051c1b30080cf10002100360090c3b300e5
:101a8000ab52e3001e003e00c872ef004212e200bb
:101a900013003600c8d2a8004012ec00d090880095
:101aa00010928000d29080000200e000020032001c
:101ab000110009000280d800e0928800e0928000c6
:101ac000b2938000c393800000004100e080490091
:101ad0000001be00f2ce880003cf88000600370068
:101ae000deb9ef00e0b9ef00262cef002068a90076
:101af0000068a90015eea900b732a8004900370018
:101b0000abd2bf0091c3b30080cf100021003600dc
:101b1000d0c5b300ab52e3001e003e00ca72ef0016
:101b20004c12e20013003600cad2a8004a12ec00a0
:101b3000d090880060928000d29080000200e00087
:101b400002003200110009000280d80010938800c2
:101b500010938000b2938000c39380000000410086
:101b6000e08049000001be0012cf880023cf88002a
:101b700006003700e2b9ef00e4b9ef00462cef00b1
:101b80002368a9000368a90015aea900b732a80010
:101b900024003700abd2bf00d1c5b30080cf100006
:101ba00020003600f0c7b300ab52e3001d003e003a
:101bb000cc72ef005612e20013003600ccd2a8001f
:101bc0005412ec00d0908800b0928000d290800037
:101bd0000200e00002003200110009000280d8007b
:101be0004093880040938000b2938000c3938000ac
:101bf00000004100e08049000001be0032cf8800b3
:101c000043cf880006003700e6b9ef00e8b9ef00df
:101c1000662cef002388a9000388a900156ea9008f
:101c2000b732a8005c013700ab52e2001c003a005a
:101c3000acd2bf00b8f2b700100ea900140ea80075
:101c4000f0c7b300b852b5000f0031002412a8004d
:101c50002612a800b8d2bf000080fb0000004000a0
:101c6000e12c210060807800b2938000c393800053
:101c700000004100e08049000001be0072ce8800f3
:101c800083ce8800040037002412a9002612a90080
:101c9000ceb9ef00d0b9ef00b732a8003d01370050
:101ca00010c0b300ab52e3001c003a00102ea90094
:101cb000142ea800acd2bf00b9f2b700f0c7b30031
:101cc000b952b5000f0031002432a8002632a80016
:101cd000b9d2bf000080fb0000004000e12c2100d1
:101ce00060807800b2938000c393800000004100c0
:101cf000e08049000001be0092ce8800a3ce88009b
:101d0000040037002432a9002632a900d2b9ef001e
:101d1000d4b9ef00b732a8001e01370020c0b300cd
:101d2000ab52e3001c003a00108ea900148ea800ec
:101d3000acd2bf00baf2b700f0c7b300ba52b500d8
:101d40000f0031002452a8002652a800bad2bf00ca
:101d50000080fb0000004000e12c21006080780042
:101d6000b2938000c393800000004100e0804900ee
:101d70000001be00b2ce8800c3ce88000400370048
:101d80002452a9002652a900d6b9ef00d8b9ef0015
:101d9000b732a800ff00370030c0b300ab52e300f9
:101da0001c003a00008ea900048ea800acd2bf002f
:101db000bbf2b700f0c7b300bb52b5000f00310053
:101dc0002472a8002672a800bbd2bf000080fb00ce
:101dd00000004000e12c210060807800b293800078
:101de000c393800000004100e08049000001be0074
:101df000d2ce8800e3ce8800040037002472a90008
:101e00002672a900dab9ef00dcb9ef00b732a800fa
:101e1000e000370040c0b300ab52e30003003a00db
:101e200010cea90014cea800da00370050c0b300cd
:101e3000ab52e30003003a0010eea90014eea80034
:101e4000d4003700abd2bf0051c1b30080cf100027
:101e50004300360090c3b300ab52e30040003e00a5
:101e6000acd2bf000080fb00e0918800abd2bf0085
:101e70000080fb0000004000e16c210060807800e1
:101e8000e0908800f293800003948000e09080004e
:101e90000cfa0700b6f90700eaf90700509388002a
:101ea000abd2bf000080fb0000004000e16c2100cd
:101eb00060807800e0908800509380001c12b5008c
:101ec0006093880015eea9000068a9002068a800aa
:101ed000c872ef00262cef00c812a800d091800035
:101ee000e29180000200e0000200320011000900cf
:101ef0000280d800c0928800e191800000928000aa
:101f0000808f50000c003200009280003c12b5001f
:101f100001e0af000020ee00f0908800f09180001a
:101f2000f29080000200e00002003200110009007f
:101f30000280d800d0928800c0928000b2938000c6
:101f4000c393800000004100e08049000001be0012
:101f5000f2ce880003cf8800b732a8008d0037008a
:101f6000abd2bf0091c3b30080cf10004300360056
:101f7000d0c5b300ab52e30040003e00acd2bf007e
:101f80000080fb0030928800abd2bf000080fb00d5
:101f900000004000e16c210060807800e090880043
:101fa0001294800023948000e0908000c5f907001f
:101fb0006ff90700a3f9070070938800abd2bf0048
:101fc0000080fb0000004000e16c21006080780090
:101fd000e0908800709380001c12b5008093880008
:101fe0000368a9002368a80015aea900ca72ef0013
:101ff000462cef00ca12a800209280003292800086
:102000000200e00002003200110009000280d80046
:10201000f09288003192800050928000808f5000b2
:102020000c003200509280004612b50001e0af0073
:102030000020ee00f090880020928000f290800056
:102040000200e00002003200110009000280d80006
:1020500000938800f0928000b2938000c3938000c8
:1020600000004100e08049000001be0012cf88005e
:1020700023cf8800b732a80046003700abd2bf009c
:10208000d1c5b30080cf100042003600f0c7b300c6
:10209000ab52e3003f003e00acd2bf000080fb002b
:1020a00080928800abd2bf000080fb00000040009f
:1020b000e16c210060807800e0908800329480001c
:1020c00043948000e09080007ef9070028f9070023
:1020d0005cf9070090938800abd2bf000080fb0042
:1020e00000004000e16c210060807800e0908800f2
:1020f000909380001c12b500a09388000388a9006b
:102100002388a800156ea900cc72ef00662cef00a2
:10211000cc12a80070928000829280000200e00041
:1021200002003200110009000280d80020938800cc
:1021300081928000a0928000808f50000c003200bd
:10214000a09280005012b50001e0af000020ee0028
:10215000f090880070928000f29080000200e00011
:1021600002003200110009000280d800309388007c
:1021700020938000b2938000c39380000000410050
:10218000e08049000001be0032cf880043cf8800c4
:10219000b732a800abf2ef003a003700c0cab30074
:1021a000a852e3000a003a0000e0ef00ad52e3005d
:1021b00003003a00a7d2bf00adf2b700030037001a
:1021c000a7d2bf00aef2b700010307002d00370011
:1021d000c0cbb300a852e3000a003a0000e0ef00d1
:1021e000af52e30003003a00a7d2bf00aff2b7003e
:1021f00003003700a7d2bf00b0f2b700fd0207000e
:1022000020003700c0ccb300a852e30007003a001a
:1022100000e0ef00b152e30003003a00a7d2bf0094
:10222000b1f2b700ec02070016003700c0cdb300d2
:10223000a852e30007003a0000e0ef00b252e300ca
:1022400003003a00a7d2bf00b2f2b700e7020700ce
:102250000c003700c0ceb300a852e30009003a00da
:1022600000e0ef00b352e30003003a00a7d2bf0042
:10227000b3f2b70003003700a7d2bf00b4f2b70033
:10228000d7020700b732af00b102070080c0b30029
:10229000b652b5009b023100b2938000c393800018
:1022a000d0938000e1938000800f5100818f59000e
:1022b000880239007df2a800b652e2000f003a0011
:1022c000120eaa00100ea900b8d2bf000080fb00b9
:1022d00000004000e12c210060807800b293800073
:1022e000c393800000004100e08049000001be006f
:1022f00072ce880083ce88007502370010c0b3000c
:10230000b652e3000f003a00122eaa00102ea900c8
:10231000b9d2bf000080fb0000004000e12c21008a
:1023200060807800b2938000c39380000000410079
:10233000e08049000001be0092ce8800a3ce880054
:102340006302370020c0b300b652e3000f003a002a
:10235000128eaa00108ea900bad2bf000080fb0026
:1023600000004000e12c210060807800b2938000e2
:10237000c393800000004100e08049000001be00de
:10238000b2ce8800c3ce88005102370030c0b300ff
:10239000b652e3000f003a00028eaa00008ea90098
:1023a000bbd2bf000080fb0000004000e12c2100f8
:1023b00060807800b2938000c393800000004100e9
:1023c000e08049000001be00d2ce8800e3ce880044
:1023d0003f02370040c0b300b652e300bd003a00f0
:1023e00010c0b300c852e3000b003a00c972ef00fe
:1023f000c832a800c0928000b2938000c3938000ce
:1024000000004100e08049000001be00f2ce8800db
:1024100003cf8800ae00370030c0b300c852e300dd
:1024200047003a00e1918000c9d2bf000080fb0064
:10243000810f500010003100c972ec00c9d2bf00fa
:102440000080fb0000004000e17c210060807800fb
:1024500030618800c0928000b2938000c3938000f6
:1024600000004100e08049000001be00f2ce88007b
:1024700003cf880031003700c872ef00e19180007f
:1024800000928000808f500005003a00c892a8009a
:10249000deb9ef00e0b9ef0040d2bf00c9f2b700eb
:1024a00000928000e1918000808f50001200360081
:1024b000c852a8003cd2bf00c9f2b700c9d2bf00c1
:1024c0000080fb0000004000e17c2100608078007b
:1024d00030618800d0928000b2938000c393800066
:1024e00000004100e08049000001be00f2ce8800fb
:1024f00003cf880011003700c872a8003cd2bf008b
:10250000c9f2b700c9d2bf000080fb000000400044
:10251000e17c21006080780030618800d0928000ea
:10252000b2938000c393800000004100e080490026
:102530000001be00f2ce880003cf8800640037009f
:1025400040c0b300c852e30019003a00c972ed0060
:10255000c9d2bf000080fb0000004000e17c2100e8
:102560006080780030618800d0928000b293800053
:10257000c393800000004100e08049000001be00dc
:10258000f2ce880003cf880001928000c9d2bf003c
:102590000080fb00810f500004003a00c852a900df
:1025a000c892a800deb9ef00e0b9ef00480037009c
:1025b00080c0b300c852e30019003a00c972ec00b1
:1025c000c9d2bf000080fb0000004000e17c210078
:1025d0006080780030618800d0928000b2938000e3
:1025e000c393800000004100e08049000001be006c
:1025f000f2ce880003cf880001928000c9d2bf00cc
:102600000080fb00810f500004003a00c872a9004e
:10261000c892a800deb9ef00e0b9ef002c00370047
:1026200000c4b300c852e3000c003a0040d2bf001f
:10263000c9f2b700c8f2a800e0928000b29380000f
:10264000c393800000004100e08049000001be000b
:10265000f2ce880003cf88001d00370000ccb30005
:10266000c852e3001a003a00c952e20010003600d6
:10267000c972ed00c9d2bf000080fb00000040001d
:10268000e17c21006080780030618800e092800069
:10269000b2938000c393800000004100e0804900b5
:1026a0000001be00f2ce880003cf8800080037008a
:1026b000c872ef00262cef000021ef002068a9006f
:1026c0000068a90015eea900deb9ef00e0b9ef003f
:1026d0007f01370050c0b300b652e300bd003a009e
:1026e00010c0b300ca52e3000b003a00cb72ef00f7
:1026f000ca32a800f0928000b2938000c393800099
:1027000000004100e08049000001be0012cf8800b7
:1027100023cf8800ae00370030c0b300ca52e300b8
:1027200047003a0031928000cbd2bf000080fb000e
:10273000810f500010003100cb72ec00cbd2bf00f3
:102740000080fb0000004000e17c210060807800f8
:1027500030628800f0928000b2938000c3938000c2
:1027600000004100e08049000001be0012cf880057
:1027700023cf880031003700ca72ef003192800009
:1027800050928000808f500005003a00ca92a80045
:10279000e2b9ef00e4b9ef004ad2bf00cbf2b700d4
:1027a0005092800031928000808f500012003600dd
:1027b000ca52a80046d2bf00cbf2b700cbd2bf00ae
:1027c0000080fb0000004000e17c21006080780078
:1027d0003062880000938000b2938000c393800031
:1027e00000004100e08049000001be0012cf8800d7
:1027f00023cf880011003700ca72a80046d2bf005c
:10280000cbf2b700cbd2bf000080fb00000040003d
:10281000e17c2100608078003062880000938000b5
:10282000b2938000c393800000004100e080490023
:102830000001be0012cf880023cf8800640037005b
:1028400040c0b300ca52e30019003a00cb72ed0059
:10285000cbd2bf000080fb0000004000e17c2100e3
:10286000608078003062880000938000b29380001e
:10287000c393800000004100e08049000001be00d9
:1028800012cf880023cf880051928000cbd2bf00a6
:102890000080fb00810f500004003a00ca52a900da
:1028a000ca92a800e2b9ef00e4b9ef00480037008f
:1028b00080c0b300ca52e30019003a00cb72ec00aa
:1028c000cbd2bf000080fb0000004000e17c210073
:1028d000608078003062880000938000b2938000ae
:1028e000c393800000004100e08049000001be0069
:1028f00012cf880023cf880051928000cbd2bf0036
:102900000080fb00810f500004003a00ca72a90049
:10291000ca92a800e2b9ef00e4b9ef002c0037003a
:1029200000c4b300ca52e3000c003a004ad2bf0010
:10293000cbf2b700caf2a80010938000b2938000d7
:10294000c393800000004100e08049000001be0008
:1029500012cf880023cf88001d00370000ccb300c1
:10296000ca52e3001a003a00cb52e20010003600cf
:10297000cb72ed00cbd2bf000080fb000000400016
:10298000e17c210060807800306288001093800034
:10299000b2938000c393800000004100e0804900b2
:1029a0000001be0012cf880023cf88000800370046
:1029b000ca72ef00462cef001421ef002368a90033
:1029c0000368a90015aea900e2b9ef00e4b9ef0071
:1029d000bf00370060c0b300b652e300bc003a004d
:1029e00010c0b300cc52e3000b003a00cd72ef00f0
:1029f000cc32a80020938000b2938000c393800063
:102a000000004100e08049000001be0032cf880094
:102a100043cf8800ae00370030c0b300cc52e30093
:102a200047003a0081928000cdd2bf000080fb00b9
:102a3000810f500010003100cd72ec00cdd2bf00ec
:102a40000080fb0000004000e17c210060807800f5
:102a50003063880020938000b2938000c39380008d
:102a600000004100e08049000001be0032cf880034
:102a700043cf880031003700cc72ef008192800094
:102a8000a0928000808f500005003a00cc92a800f0
:102a9000e6b9ef00e8b9ef0054d2bf00cdf2b700bd
:102aa000a092800081928000808f5000120036003a
:102ab000cc52a80050d2bf00cdf2b700cdd2bf009b
:102ac0000080fb0000004000e17c21006080780075
:102ad0003063880030938000b2938000c3938000fd
:102ae00000004100e08049000001be0032cf8800b4
:102af00043cf880011003700cc72a80050d2bf002d
:102b0000cdf2b700cdd2bf000080fb000000400036
:102b1000e17c210060807800306388003093800081
:102b2000b2938000c393800000004100e080490020
:102b30000001be0032cf880043cf88006400370018
:102b400040c0b300cc52e30019003a00cd72ed0052
:102b5000cdd2bf000080fb0000004000e17c2100de
:102b6000608078003063880030938000b2938000ea
:102b7000c393800000004100e08049000001be00d6
:102b800032cf880043cf8800a1928000cdd2bf0011
:102b90000080fb00810f500004003a00cc52a900d5
:102ba000cc92a800e6b9ef00e8b9ef004800370082
:102bb00080c0b300cc52e30019003a00cd72ec00a3
:102bc000cdd2bf000080fb0000004000e17c21006e
:102bd000608078003063880030938000b29380007a
:102be000c393800000004100e08049000001be0066
:102bf00032cf880043cf8800a1928000cdd2bf00a1
:102c00000080fb00810f500004003a00cc72a90044
:102c1000cc92a800e6b9ef00e8b9ef002c0037002d
:102c200000c4b300cc52e3000c003a0054d2bf0001
:102c3000cdf2b700ccf2a80040938000b2938000a0
:102c4000c393800000004100e08049000001be0005
:102c500032cf880043cf88001d00370000ccb3007e
:102c6000cc52e3001a003a00cd52e20010003600c8
:102c7000cd72ed00cdd2bf000080fb00000040000f
:102c8000e17c210060807800306388004093800000
:102c9000b2938000c393800000004100e0804900af
:102ca0000001be0032cf880043cf88000800370003
:102cb000cc72ef00662cef001821ef002388a900ea
:102cc0000388a900156ea900e6b9ef00e8b9ef0086
:102cd0001f00070079f2ae00090037007632ef00de
:102ce0007832ef000621ef000a21ef002432ef00d6
:102cf0000080eb00e19c21000f00090080187800a3
:102d00000600370079f2ae00040037007632ef009b
:102d10007832ef000621ef000a21ef00a5d2bf00b4
:102d2000a652e300090032000188af000700370017
:102d3000a672ec00a6d2bf000080fb00e1ae21002d
:102d400060c078000080fb0020118800f7f9370090
:102d5000b6f2ef007df2a800b572ef0070c0b300cc
:102d6000b552e30018003e00b5d2bf000080fb0062
:102d7000c200dd00e09c2100008040001000be0089
:102d80000001be00d0938000e1938000800f5100cd
:102d9000818f59000a003100b5d2bf000080fb00ce
:102da000c200dd00e09c2100008040001000be0059
:102db000d0938800e1938800b5d2bf00b6f2b70087
:102dc000b572ec00e5ff3900b732a900000006003b
:102dd000adf2ef0000000600b1f2ef0000000600c7
:102de000b3f2ef00b4f2ef0000000600b2f2ef0021
:102df0000000060070c0b300af52e3000a003a00c2
:102e0000b0d2bf000080fb0000928800b0d2bf00ab
:102e10000080fb0050928800b0d2bf000080fb0011
:102e2000a0928800bb00370000c1b300af52e3009e
:102e300009003a00b072ec000200200003382400c0
:102e4000b0d2bf001ef6070086f50700f093880099
:102e500001948800af00370010c1b300af52e30007
:102e600006003a00b0d2bf000080fb00323b2000d9
:102e70000200b800d0918800a600370020c1b3003e
:102e8000af52e30006003a00b0d2bf000080fb0062
:102e9000323b20000200b800f09188009d0037000e
:102ea00030c1b300af52e30006003a00b0d2bf0019
:102eb0000080fb00323b20000200b8001092880026
:102ec00094003700a0c1b300af52e30009003a00fc
:102ed000b072ec000200200003382400b0d2bf0022
:102ee000f7f507005ff5070010948800219488002b
:102ef00088003700b0c1b300af52e30006003a00cb
:102f0000b0d2bf000080fb00323b20000200b800be
:102f1000209288007f003700c0c1b300af52e300a9
:102f200006003a00b0d2bf000080fb00323b200018
:102f30000200b8004092880076003700d0c1b3008c
:102f4000af52e30006003a00b0d2bf000080fb00a1
:102f5000323b20000200b800609288006d0037000c
:102f6000e0c1b300af52e30005003a00b0d2bf00a9
:102f7000bcf2b700b0d2bf00bdf2b70065003700a9
:102f800040c2b300af52e30009003a00b072ec0057
:102f90000200200003382400b0d2bf00c8f50700ab
:102fa00030f50700309488004194880059003700bc
:102fb00050c2b300af52e30006003a00b0d2bf00e7
:102fc0000080fb00323b20000200b80070928800b5
:102fd0005000370060c2b300af52e30006003a0071
:102fe000b0d2bf000080fb00323b20000200b800de
:102ff000909288004700370070c2b300af52e300e0
:1030000006003a00b0d2bf000080fb00323b200037
:103010000200b800b09288003e00370020c4b30020
:10302000af52e30004003a00b052e20001003a005f
:103030003a00070037003700b0c7b300af52e300d3
:103040001f003a000c003700262cef00462cef0042
:10305000662cef0015eea90015aea900156ea900ab
:10306000c872ef00ca72ef00cc72ef002068a900ae
:103070002368a9002388a9002432ef002632ef003c
:10308000b732a800b572ef0070c0b300b552e300cc
:103090000a003e00b5d2bf000080fb00c200dd0088
:1030a000e09c210000814000f0ff2f00f1ff2f0085
:1030b0000089be00b572ec00f3ff3900150037003f
:1030c000e0c7b300af52e30012003a00a572ec0073
:1030d000a5d2bf000080fb00c20b2000e1ae2100a2
:1030e00002f07800a572ec00a5d2bf000080fb00c2
:1030f000e2072000e1ae210002f07800a572ec00aa
:10310000a5d2bf000081fb00e1ae2100b0d2bf001c
:1031100000f17800aff2ef0000000600100ea900e9
:10312000140ea900102ea900142ea900108ea900bb
:10313000148ea900008ea900048ea90010cea9004b
:1031400014cea90010eea90014eea9002632ef005b
:103150002432ef00b732a800b872ef00b972ef0066
:10316000ba72ef00bb72ef00bc72ef00bd72ef00ed
:10317000be72ef00bf72ef00b572ef0070c0b30017
:10318000b552e3000a003e00b5d2bf000080fb004c
:10319000c200dd00e09c210000814000f0ff2f0014
:1031a000f1ff2f000089be00b572ec00f3ff39007b
:1031b000262cef00462cef00662cef0011eea90044
:1031c00015eea90011aea90015aea900116ea90057
:1031d000156ea900c872ef00ca72ef00cc72ef0042
:1031e0002068a9002368a9002388a9000000060020
:1031f000ceb2ef00a0c72500809688005098250029
:103200009096880040812500a0968800906a25004d
:10321000b096880030542500c0968800303e2500c6
:10322000d096880090282500e0968800501325004d
:10323000f096880060fe240000978800c0e9240012
:103240001097880080d524002097880090c1240022
:1032500030978800f0ad240040978800a09a2400a1
:1032600050978800a087240060978800f07424009d
:103270007097880090622400809788008050240016
:1032800090978800b03e2400a0978800302d24003d
:10329000b0978800f01b2400c0978800000b240022
:1032a000d097880050fa2300e0978800e0e92300d7
:1032b000f0978800c0d9230000988800e0c9230057
:1032c0001098880040ba230020988800e0aa2300c4
:1032d00030988800c09b230040988800e08c230031
:1032e00050988800307e230060988800d06f2300bb
:1032f00070988800a061230080988800b053230054
:1033000090988800f0452300a0988800703823002a
:10331000b0988800202b2300c0988800101e23003e
:10332000d098880040112300e09888009004230082
:10333000f098880020f8220000998800e0eb220035
:1033400010998800d0df220020998800f0d3220055
:103350003099880050c8220040998800d0bc2200d3
:103360005099880080b122006099880070a62200e0
:1033700070998800809b220080998800c09022006c
:103380009099880020862200a0998800c07b2200a6
:10339000b099880080712200c0998800606722007f
:1033a000d0998800805d2200e0998800c0532200f7
:1033b000f0998800204a2200009a8800b04022003c
:1033c000109a880060372200209a8800402e220040
:1033d000309a880040252200409a8800601c220014
:1033e000509a8800b0132200609a8800200b2200b7
:1033f000709a8800b0022200809a880060fa21004a
:10340000909a880040f22100a09a880030ea2100ba
:10341000b09a880050e22100c09a880090da21001a
:10342000d09a8800e0d22100e09a880060cb210089
:10343000f09a8800f0c32100009b8800b0bc2100f6
:10344000109b880080b52100209b880080ae210061
:10345000309b880090a72100409b8800b0a02100ed
:10346000509b8800009a2100609b88006093210097
:10347000709b8800e08c2100809b88008086210062
:10348000909b880030802100a09b8800007a21005a
:10349000b09b8800f0732100c09b8800f06d210074
:1034a000d09b880000682100e09b880040622100da
:1034b000f09b8800805c2100009c8800e056210081
:1034c000109c880060512100209c8800f04b210056
:1034d000309c880090462100409c8800504121008b
:1034e000509c8800203c2100609c880010372100ff
:1034f000709c880010322100809c8800202d2100c3
:10350000909c880040282100a09c880080232100f6
:10351000b09c8800d01e2100c09c8800301a210079
:10352000d09c8800a0152100e09c8800201121007b
:10353000f09c8800c00c2100009d880070082100cc
:10354000109d880020042100209d8800f0ff2000ad
:10355000309d8800d0fb2000409d8800c0f72000ef
:10356000509d8800d0f32000609d8800e0ef20008f
:10357000709d880000ec2000809d880030e82000cd
:10358000909d880070e42000a09d8800c0e020008d
:10359000b09d880020dd2000c09d880090d92000cb
:1035a000d09d880010d62000e09d8800a0d2200089
:1035b000f09d880040cf2000009e8800e0cb2000d6
:1035c000109e8800a0c82000209e880060c52000b2
:1035d000309e880030c22000409e880010bf20002e
:1035e000509e880000bc2000609e8800ceb3ef0093
:1035f000302c2a00809e880060a42900909e8800bc
:1036000020632900a09e8800a0232900b09e880086
:10361000d0e52800c09e8800a0a92800d09e880080
:10362000006f2800e09e8800f0352800f09e88009a
:1036300070fe2700009f880050c82700109f880058
:10364000b0932700209f880070602700309f88007b
:10365000802e2700409f8800f0fd2600509f8800a4
:10366000a0ce2600609f8800a0a02600709f880042
:10367000c0732600809f880020482600909f880005
:10368000a01d2600a09f880040f42500b09f880060
:10369000f0cb2500c09f8800c0a42500d09f8800e3
:1036a000907e2500e09f880060592500f09f8800eb
:1036b0003035250000a088000012250010a08800e9
:1036c000b0ef240020a0880050ce240030a0880055
:1036d000c0ad240040a08800208e240050a08800a7
:1036e000506f240060a088005051240070a0880012
:1036f0002034240080a08800b017240090a0880007
:1037000000fc2300a0a0880000e12300b0a08800f6
:10371000d0c62300c0a0880040ad2300d0a0880000
:1037200060942300e0a08800207c2300f0a08800a3
:103730009064230000a18800a04d230010a1880000
:103740004037230020a188008021230030a1880079
:10375000500c230040a18800b0f7220050a188003f
:10376000a0e3220060a1880020d0220070a1880080
:1037700010bd220080a1880090aa220090a188009c
:1037800080982200a0a18800f0862200b0a18800c5
:10379000e0752200c0a1880030652200d0a1880019
:1037a00000552200e0a1880040452200f0a18800d9
:1037b000e035220000a28800f026220010a2880036
:1037c0006018220020a28800300a220030a288005f
:1037d00060fc210040a28800f0ee210050a2880089
:1037e000e0e1210060a2880020d5210070a28800bd
:1037f000c0c8210080a28800b0bc210090a288002f
:10380000f0b02100a0a2880080a52100b0a288000d
:10381000509a2100c0a28800808f2100d0a2880089
:10382000f0842100e0a28800b07a2100f0a2880094
:10383000a070210000a38800f066210010a388007a
:10384000705d210020a388003054210030a388003f
:10385000304b210040a388007042210050a3880013
:10386000f039210060a38800a031210070a38800f6
:103870009029210080a38800b021210090a3880016
:10388000101a2100a0a3880090122100b0a3880084
:10389000500b2100c0a3880040042100d0a3880061
:1038a00060fd2000e0a38800b0f62000f0a38800af
:1038b00030f0200000a48800d0e9200010a4880087
:1038c000a0e3200020a48800a0dd200030a4880010
:1038d000c0d7200040a4880010d2200050a4880047
:1038e00080cc200060a4880020c7200070a488003d
:1038f000e0c1200080a48800c0bc200090a4880003
:10390000c0b72000a0a48800e0b22000b0a48800c6
:1039100030ae2000c0a4880090a92000d0a4880068
:1039200010a52000e0a48800b0a02000f0a488002a
:10393000809c200000a588005098200010a58800d9
:103940005094200020a588006090200030a58800b9
:10395000908c200040a58800e088200050a58800b9
:103960004085200060a58800c081200070a58800e7
:10397000507e200080a58800f07a200090a5880065
:10398000b0772000a0a5880090742000b0a5880022
:1039900070712000c0a58800706e2000d0a588003e
:1039a000906b2000e0a58800b0682000f0a588009a
:1039b000f065200000a688004063200010a6880063
:1039c000a060200020a68800105e200030a688009d
:1039d000905b200040a688003059200050a6880047
:1039e000d056200060a68800b572ef00f0c7b30083
:1039f000b552e3000e003e00b5d2bf000080fb00d0
:103a000000004000e13c2100608078004300de00bf
:103a1000512b2100914078008180fb008180400083
:103a2000e23c210080307900b572ec00efff3900f4
:103a30000000060030b62f00d0b7880070d42e00ea
:103a4000e0b7880060ff2d00f0b7880040362d00f9
:103a500000b8880070782c0010b8880040c52b0092
:103a600020b88800201c2b0030b88800807c2a00f9
:103a700040b88800d0e5290050b88800a057290038
:103a800060b8880060d1280070b88800b052280063
:103a900080b8880020db270090b88800406a2700a3
:103aa000a0b88800b0ff2600b0b88800209b260090
:103ab000c0b88800303c2600d0b88800a0e22500bd
:103ac000e0b88800108e2500f0b88800403e250040
:103ad00000b98800f0f2240010b98800d0ab2400af
:103ae00020b98800b068240030b98800502924002b
:103af00040b9880090ed230050b9880020b523001c
:103b000060b98800d07f230070b98800904d2300f1
:103b100080b98800201e230090b9880050f122004f
:103b2000a0b9880000c72200b0b98800209f2200f9
:103b3000c0b9880070792200d0b98800e055220011
:103b4000e0b9880060342200f0b98800b014220087
:103b500000ba8800c0f6210010ba880090da21006f
:103b600020ba8800f0bf210030ba8800c0a621002a
:103b700040ba8800108f210050ba8800a078210038
:103b800060ba88008063210070ba8800904f2100dd
:103b900080ba8800c03c210090ba8800f02a210039
:103ba000a0ba8800301a2100b0ba8800500a21005b
:103bb000c0ba880060fb2000d0ba880040ed200029
:103bc000e0ba8800f0df2000f0ba880060d320005f
:103bd00000bb880080c7200010bb880050bc2000bc
:103be00020bb8800c0b1200030bb8800c0a72000e7
:103bf00040bb8800609e200050bb8800809520005c
:103c000060bb8800108d200070bb880030852000cc
:103c100080bb8800b07d200090bb8800a07620008b
:103c2000a0bb880000702000b0bb8800b0692000f5
:103c3000c0bb8800c0632000d0bb8800305e20007d
:103c4000e0bb8800e0582000f0bb8800e053200073
:103c500000bc8800304f200010bc8800c04a200003
:103c600020bc88009046200030bc88009042200094
:103c700040bc8800e03e200050bc8800503b200043
:103c800060bc88000038200070bc8800e034200050
:103c900080bc8800e031200090bc8800102f2000fc
:103ca000a0bc8800702c2000b0bc8800f029200047
:103cb000c0bc880090272000d0bc88006025200070
:103cc000e0bc880040232000f0bc88005021200088
:103cd00000bd8800701f200010bd8800b01d2000ae
:103ce00020bd8800001c200030bd8800701a200014
:103cf00040bd8800f018200050bd880090172000bb
:103d000060bd88004016200070bd880000152000ae
:103d100080bd8800d013200090bd8800b012200024
:103d2000a0bd8800a0112000b0bd8800a010200018
:103d3000c0bd8800b00f2000d0bd8800d00e20008c
:103d4000e0bd8800000e2000f0bd8800300d20008e
:103d500000be8800800c200010be8800c00b200030
:103d600020be8800200b200030be8800800a200082
:103d700040be8800e009200050be880050092000a5
:103d800060be8800000006000004200070be8800ad
:103d9000009c2f0070c688004004200080be880070
:103da000c09b2f0080c688007004200090be880051
:103db000909b2f0090c68800b0042000a0be880011
:103dc000509b2f00a0c6880000052000b0be8800d0
:103dd000009b2f00b0c6880040052000c0be8800b0
:103de000c09a2f00c0c6880090052000d0be880071
:103df000709a2f00d0c68800e0052000e0be880041
:103e0000209a2f00e0c6880030062000f0be88000f
:103e1000d0992f00f0c688008006200000bf8800df
:103e200080992f0000c78800e006200010bf88009e
:103e300020992f0010c788004007200020bf88006d
:103e4000c0982f0020c78800b007200030bf88002e
:103e500050982f0030c788002008200040bf8800fd
:103e6000e0972f0040c788009008200050bf8800ce
:103e700070972f0050c788001009200060bf88008d
:103e8000f0962f0060c788009009200070bf88005e
:103e900070962f0070c78800100a200080bf88002d
:103ea000f0952f0080c78800a00a200090bf8800ee
:103eb00060952f0090c78800400b2000a0bf8800ad
:103ec000c0942f00a0c78800e00b2000b0bf88007e
:103ed00020942f00b0c78800900c2000c0bf88003d
:103ee00070932f00c0c78800400d2000d0bf88000d
:103ef000c0922f00d0c78800000e2000e0bf8800cd
:103f000000922f00e0c78800c00e2000f0bf88009c
:103f100040912f00f0c78800900f200000c088005b
:103f200070902f0000c888007010200010c088001a
:103f3000908f2f0010c888006011200020c08800da
:103f4000a08e2f0020c888005012200030c08800aa
:103f5000b08d2f0030c888006013200040c088005a
:103f6000a08c2f0040c888007014200050c088002a
:103f7000908b2f0050c88800a015200060c08800da
:103f8000608a2f0060c88800d016200070c08800aa
:103f900030892f0070c888001018200080c0880069
:103fa000f0872f0080c888007019200090c088001a
:103fb00090862f0090c88800d01a2000a0c08800ea
:103fc00030852f00a0c88800501c2000b0c0880099
:103fd000b0832f00b0c88800f01d2000c0c088004a
:103fe00010822f00c0c88800a01f2000d0c0880009
:103ff00060802f00d0c8880060212000e0c08800c9
:10400000a07e2f00e0c8880040232000f0c0880078
:10401000c07c2f00f0c888003025200000c1880037
:10402000d07a2f0000c988005027200010c18800d6
:10403000b0782f0010c988008029200020c1880096
:1040400080762f0020c98800d02b200030c1880046
:1040500030742f0030c98800402e200040c18800f5
:10406000c0712f0040c98800d030200050c18800a6
:10407000306f2f0050c988009033200060c1880045
:10408000706c2f0060c988007036200070c18800f5
:1040900090692f0070c988008039200080c1880095
:1040a00080662f0080c98800b03c200090c1880045
:1040b00050632f0090c9880010402000a0c18800e4
:1040c000f05f2f00a0c98800b0432000b0c1880075
:1040d000505c2f00b0c9880070472000c0c1880024
:1040e00090582f00c0c98800704b2000d0c18800b4
:1040f00090542f00d0c98800b04f2000e0c1880044
:1041000050502f00e0c9880020542000f0c18800e2
:10411000e04b2f00f0c98800d058200000c2880072
:1041200030472f0000ca8800d05d200010c28800f0
:1041300030422f0010ca88000063200020c288008f
:10414000003d2f0020ca88009068200030c28800ff
:1041500070372f0030ca8800706e200040c288007f
:1041600090312f0040ca88009074200050c288000f
:10417000702b2f0050ca8800207b200060c288006e
:10418000e0242f0060ca88000082200070c28800ee
:10419000001e2f0070ca88004089200080c288005d
:1041a000c0162f0080ca8800f090200090c28800be
:1041b000100f2f0090ca880000992000a0c288002c
:1041c00000072f00a0ca880090a12000b0c288007c
:1041d00070fe2e00b0ca8800a0aa2000c0c28800cd
:1041e00060f52e00c0ca880020b42000d0c288002c
:1041f000e0eb2e00d0ca880030be2000e0c288006c
:10420000d0e12e00e0ca8800d0c82000f0c28800ab
:1042100030d72e00f0ca880010d4200000c38800d8
:10422000f0cb2e0000cb8800f0df200010c3880008
:1042300010c02e0010cb880070ec200020c3880036
:1042400090b32e0020cb8800a0f9200030c3880056
:1042500060a62e0030cb8800a007210040c3880054
:1042600060982e0040cb88005016210050c3880073
:10427000b0892e0050cb8800e025210060c3880063
:10428000207a2e0060cb88005036210070c3880051
:10429000b0692e0070cb8800b047210080c3880031
:1042a00050582e0080cb8800005a210090c388000f
:1042b00000462e0090cb8800506d2100a0c38800de
:1042c000b0322e00a0cb8800c0812100b0c388008e
:1042d000401e2e00b0cb880050972100c0c388003c
:1042e000b0082e00c0cb880010ae2100d0c38800db
:1042f000f0f12d00d0cb880020c62100e0c388005b
:10430000e0d92d00e0cb880080df2100f0c38800d9
:1043100080c02d00f0cb880050fa210000c4880036
:10432000b0a52d0000cc8800a016220010c4880083
:1043300060892d0010cc88008034220020c48800c1
:10434000806b2d0020cc88001054220030c48800df
:10435000f04b2d0030cc88006075220040c48800ee
:10436000a02a2d0040cc88009098220050c48800dc
:1043700070072d0050cc8800b0bd220060c48800ba
:1043800050e22c0060cc8800f0e4220070c4880069
:1043900010bb2c0070cc8800600e230080c4880005
:1043a000a0912c0080cc8800103a230090c4880093
:1043b000f0652c0090cc880040682300a0c48800e1
:1043c000c0372c00a0cc880000992300b0c488001e
:1043d00000072c00b0cc880080cc2300c0c488002b
:1043e00080d32b00c0cc8800e0022400d0c4880019
:1043f000209d2b00d0cc8800403c2400e0c48800e5
:10440000c0632b00e0cc8800e0782400f0c4880072
:1044100020272b00f0cc8800e0b8240000c58800dd
:1044200020e72a0000cd880070fc240010c5880019
:1044300090a32a0010cd8800c043250020c5880025
:10444000405c2a0020cd8800208f250030c58800e0
:10445000e0102a0030cd8800b0de250040c588007d
:1044600050c1290040cd8800b032260050c58800d8
:10447000506d290050cd8800608b260060c58800f3
:10448000a014290060cd880000e9260070c58800ce
:1044900000b7280070cd8800e04b270080c5880059
:1044a0002054280080cd880050b4270090c5880093
:1044b000b0eb270090cd880090222800a0c588008e
:1044c000707d2700a0cd8800f0962800b0c5880038
:1044d00010092700b0cd8800e0112900c0c5880070
:1044e000208e2600c0cd8800b0932900d0c588005a
:1044f000500c2600d0cd8800b01c2a00e0c58800f2
:1045000050832500e0cd880070ad2a00f0c58800fa
:1045100090f22400f0cd880030462b0000c68800c1
:10452000d059240000ce880090e72b0010c68800e8
:1045300070b8230010ce8800e0912c0020c68800bf
:10454000200e230020ce8800c0452d0030c68800f4
:10455000405a220030ce8800b0032e0040c68800aa
:10456000509c210040ce880040cc2e0050c68800d0
:10457000c0d3200050ce880000a02f0060c6880065
:104580000004200060ce8800b572ef00f0c7b300d1
:10459000b552e3001a003e00b5d2bf000080fb0018
:1045a00000004000e17c2100608078004600de00d1
:1045b000512b2100914078008180fb0081804000d8
:1045c000e27c210080307900b5d2bf000080fb0082
:1045d00000004000e18c2100608078004600de0091
:1045e000512b2100914078008180fb0081804000a8
:1045f000e28c210080307900b572ec00e3ff3900d5
:0846000000000600ffff370077
:020000040000fa
:104608001a120000080000008000000022120000ba
:104618005400000080000000761200002c0000000a
:1046280080000000a21200002c00000080000000a2
:10463800ce1200000007000080000000ce19000024
:104648002000000080000000ee1900000a020000af
:084658008000000000000000da
:00000001FF
